:030000000247BBF9
:0C47BB0078FFE4F6D8FD75816102480229
:101D29000A53746172743A20004950436F6E6E65AC
:101D390063745245510A004950436F6E6E6563746E
:101D4900003E432C562C52432CC0E4E0EFF2E5F060
:101D590020D1E8EDEAEEEC49500A003E432C4D4112
:101D6900432C25303262583A25303262583A2530B0
:101D79003262583A25303262583A25303262583A3E
:101D890025303262582C4D414320E0E4F0E5F10A58
:101D9900003E432C5645522C20332E3120EEF220A2
:101DA90025732025732CC2E5F0F1E8FF2049502066
:101DB900ECEEE4F3EBFF0A004E6F7620303320326D
:101DC9003030370030383A35313A3033003E432C21
:101DD9004C442C50524F473A2020202020202020CC
:101DE90020202020202020202020202020202020EA
:101DF90020202020202020202020202020202020DA
:101E090020202020202020202020202020202020C9
:101E1900202020202020202020202020202CC4E049
:101E2900F2E020EFF0EEF8E8E2EAE828F4E0E9EB86
:101E3900290A003E2A2C312CCEF1EDEEE2EDFBE52C
:101E490020EFE0F0E0ECE5F2F0FB20F1E5F2E5E26D
:101E5900EEE3EE20E8EDF2E5F0F4E5E9F1E00A0061
:101E69003E412C4130312C2562752E2562752E2577
:101E790062752E2562752C495020E0E4F0E5F120C9
:101E8900E0E4E0EFF2E5F0E00A003E412C413032B7
:101E99002C2562752E2562752E2562752E25627593
:101EA9002C495020E0E4F0E5F120EEF1ED2E20F18F
:101EB900E5F0E2E5F0E00A003E412C4130332C2503
:101EC90062752E2562752E2562752E2562752C493F
:101ED9005020E0E4F0E5F120F0E5E72E20F1E5F00F
:101EE900E2E5F0E00A003E412C4130342C256275D0
:101EF9002E2562752E2562752E2562752CCCE0F192
:101F0900EAE020F1E5F2E80A003E412C4130352CA7
:101F19002562752E2562752E2562752E2562752C12
:101F2900D8EBFEE70A003E532C4130362C2562756A
:101F39002CC2F0E5ECFF20EEE6E8E42E20EAE2E828
:101F4900F2E0EDF6E8E820282A3130ECF1290A0020
:101F59003E2A2C312CC4EEEF2E20EFE0F0E0ECE528
:101F6900F2F0FB20F1E5F2E5E2EEE3EE20E8EDF236
:101F7900E5F0F4E5E9F1E00A003E422C5330312C5A
:101F89002562752CC6E4E0F2FC20E7E0EFF0EEF103
:101F9900E020F1EEE5E4E8EDE5EDE8FF20EEF220E2
:101FA900F1E5F0E2E5F0E00A003E422C5330322C34
:101FB9002562752CCEE1ECE5ED20F120F1E5F0E2AA
:101FC900E5F0EEEC20E1E5E720EAE2E8F2E0EDF603
:101FD900E8E90A003E422C5330332C2562752CCF98
:101FE900E5F0E5E7E0EFF3F1EA20EFF0E820EFEEC6
:101FF900F2E5F0E520F1E2FFE7E820F120F1E5F074
:10200900E2E5F0EEEC0A003E422C5330342C256216
:10201900752CCDE5F220EFE5F0E5E4E0F7E820E402
:10202900E8E0E3EDEEF1F2E8EAE820E220F1E5F09C
:10203900E2E5F00A003E422C5330352C2562752C1E
:10204900CAE0EDE0EB20F8E8F0EEEAEEE2E5F8E0D0
:10205900F2E5EBFCEDEEE3EE20EEE1ECE5EDE00A76
:10206900003E532C5330362C2530326258253032FD
:102079006258253032625825303262582530326232
:102089005825303262582C4D414320E0E4F0E5F107
:1020990020F8E8F0EEEAEEE2E5F8E0F2E5EBFCED37
:1020A900EEE3EE20EEE1ECE5EDE00A003E454E44BC
:1020B9000A0044756D7058202020202030302030CF
:1020C9003120303220303320303420303520303642
:1020D900203037203038203039203041203042201C
:1020E90030432030442030452030460A003A200051
:1020F9000A0044756D7044202020202030302030A3
:102109003120303220303320303420303520303601
:1021190020303720303820303920304120304220DB
:1021290030432030442030452030460A0045727241
:10213900206B657900526420656570726F6D0A00C5
:102149005264204D454D0A00526420436F64650A6C
:102159000044656275674950204F4E0A0044656224
:1021690075674950204F46460A00446562756755B0
:10217900736572204F6E0A00446562756755736511
:1021890072204F46460A0044656275674D736720A1
:102199004F6E0A0044656275674D7367204F464666
:1021A9000A00436F6E666967206C6F636B210A00D2
:1021B900577220656570726F6D0A002053617665EC
:1021C90020656570726F6D210A00457272204D415C
:1021D9004321004C6F61643E3E002A003C4130318E
:1021E9003D003C4130323D003C4130333D003C41F3
:1021F90030343D003C4130353D003C4130363D00F6
:102209004E4F4950004C494E4B434F4E5452005487
:1022190052415353004652004E4F4C494E4B0049D0
:102229004E49004E4F4449414700003C21003C5370
:1022390030313D003C5330323D003C5330333D009A
:102249003C5330343D003C5330353D003C5330362F
:102259003D00FF2209FF220EFF2218FF221EFF2246
:0A22690021FF2228FF222CFF223360
:06526300015E00015C0089
:1051CD00C2AFC28E438910758BFF758DB7D2ABD22E
:0451DD008ED2AF229D
:03001B000244CDCF
:1044CD00C0E0C083C082C0D0C2AFC28E758BFF75F5
:1044DD008DB720160675A61E75A6E1055CD212E5F0
:1044ED005E6002055EE55DD394014002155D0561D8
:1044FD00E561540F7050D21DE561543F701AD21012
:10450D00906EC7E0601204F0E0D394B4400A90803E
:10451D00007480F0C2AF80FE906EC2E0600204F0C5
:10452D0090693EE0600214F0906EC8E0D3940140B3
:10453D0003E014F0301502055FE560D39464400488
:10454D00D21680020560E55BD394014002155BD263
:0C455D008ED2AFD0D0D082D083D0E0321C
:1017B000C21A7D027C007F0712517F8F26E52664C6
:1017C0006060097D017F601250D2D21AE4FDFC7F77
:1017D0000B12517F8F26E52630E6097D04E4FF12C7
:1017E00050F6D21A7D017C007F0712517F8F26E5CB
:1017F000267008FD7FFF1250D2D21A301A031260F1
:1018000000C2AFC288C2A8C2AA758900124569D2B7
:10181000AF906B867403F0A374CCF0E4906B85F00A
:10182000123D68EF600312300E1233B3C216124D30
:101830005F906B92E0C3940350037403F0D21AC21A
:101840001CC21BD293201A077E1D7F29123E4EE434
:10185000906DB2F01251CDC2AFA37408F0906AF14E
:101860007424F0E4A3F0906B7BE0906AF3F0906B4B
:101870007CE0906AF4F0906B7DE0906AF5F0906BFC
:101880007EE0906AF6F0906B7FE0906AF7F0906BE4
:1018900080E0906AF8F0755D01E4906DB4F0C217D5
:1018A000C218D2AF75A70775A61E75A6E11250AB78
:1018B000201A19AF267E007D031240EDE4FF12448A
:1018C000237E6B7FB2E4FB7D0112429D906EC7E0E8
:1018D00060037401F0E490693EF0A37455F0A374C2
:1018E00081F0E4F55FE4F56090693EE07003122555
:1018F000CF906EC8E0B401119080007410F0E490B5
:101900006EC8F0D21AD21BD21C908008E0F52630A7
:10191000E405D2177410F0E52630E508D21990805E
:10192000087420F0E52630E608D21890800874404C
:10193000F0E55FD394034023908002E4F0908001AF
:10194000F0908000F0E55FD39406400FE4F55FC2AD
:1019500013906DB4F0755D01124D5F9080A0E07042
:1019600003124B509080B8E07003124BCA9080D0A5
:10197000E07003124C44908000E070133017101296
:101980003C64906B6EEFF0D3940040031208E79034
:101990008002E07006908000E06005D2150218E534
:1019A000C215E4F55F90693EE060030218E5301966
:1019B000121239E5906B6EEFF0D394004005E0FF12
:1019C000125218201803021B3F123701906B6EEF62
:1019D000F070030218E5906BB2E054BF247F7003EF
:1019E000021AA2147003021A7A24026003021AD5A2
:1019F000201A077E1D7F32123E4E301E7420137156
:101A0000906B8AE0FF7006906B8EE06055906EBE22
:101A1000E0FEB50722A3E0FF906B8BE0B5071890BE
:101A20006EC0E0FF906B8CE0B5070C906EC1E0FFDC
:101A3000906B8DE06F602B906B8EE06E7033906ECC
:101A4000BFE0FF906B8FE0B50727906EC0E0FF907E
:101A50006B90E0B5071B906EC1E0FF906B91E0B515
:101A6000070F906DB47401F0120021755D01021B27
:101A70003F906EBE74FFF0021B3F906EC7E06003A4
:101A80007401F0906EB6E0FF906BB4E06F600302FB
:101A90001B3F906EB6E004F0E4F55D906DB2F0028D
:101AA0001B3F301303021B3F906B81E07003021851
:101AB000E5125278D213E4F55D906DB2F0906EC2EB
:101AC00004F0E4906EB5F0A3F0201A737E1D7F4001
:101AD000123E4E806A906EC7E060037401F03013CE
:101AE00052906BB2E020E74B906BB4E0FF906EB584
:101AF000E0FE6F600D906EBDE07007EE146F703FFA
:101B00008013906EB5E004F0906B6EE0FFD3940408
:101B10004003124E4690683A7482F0A37401F0902C
:101B20006BB4E090683CF07E687F3A7D03124AD542
:101B30000218E5301E09201306906EBE74FFF020D7
:101B40001303021BF4E55D706B124F79EF60207E8A
:101B50006C7FB2906CB3E02404FD124AD5906EBD48
:101B6000E060030218E5906B92E0F55D0218E590E5
:101B70006EC2E0D3943C403C906EBDE07036906EF7
:101B8000C204F0906AF0E0702B125259E4906CB2EB
:101B9000F0A37412F0906EB6E0906CB4F0A374FDF4
:101BA000F090694163A201906CB663A2017F1212AA
:101BB00032DC809B12524EEF601590683A7483F0CD
:101BC000E4A3F07E687F3A7D02124AD50218E5E56B
:101BD0005D640160030218E5906DB2E004F0E0C3BB
:101BE00094055003021B4FC213E4906DB4F0120031
:101BF000210218E5E55D640160030218E5906DB40B
:101C0000E014604024FE603C147003021CDC2404D9
:101C100060030218E5E4F55F201E13906DB47404B0
:101C2000F0906DB2E05401F0755D010218E5E490AA
:101C30006DB4F0906DB204F0755DC8906EBE74FF27
:101C4000F00218E5906EBEE07003021CCB906CB2FF
:101C50007480F0906CB47401F0E4A3F0A304F0A3DA
:101C60007430F0A3747BF0E4F52674B92526F58270
:101C7000E4346CF583747DF074BA2526F582E4347F
:101C80006CF583E4F0E5262407906CB3F07C6E7D60
:101C9000BE906B86E0FAA3E0FB7F021249517E6C96
:101CA0007FB2E5262409FD124AD5906EBDE0601B87
:101CB000125278D213E4F55D906DB2F0906EC204CA
:101CC000F0E4906EB5F0A3F00218E5906DB47404E2
:101CD000F0906B92E02432F55D0218E5908002747A
:101CE00010F0755D03906DB2E06401FFF0906DB48B
:101CF0007401F0EF7019906B8EE06013FCA3E0FDAF
:101D0000A3E0FEA3E0FF906EBE122A260218E59023
:101D10006B8AE0FCA3E0FDA3E0FEA3E0FF906EBEB3
:081D2000122A260218E580FEDC
:011D28002298
:1008E700906BB3E0B444047F0180027F00906BB249
:1008F700E0B447047E0180027E00EE5F604A906BA1
:100907007BE0906BB4F0906B7CE0906BB5F0906BF4
:100917007DE0906BB6F0906B7EE0906BB7F0906BDC
:100927007FE0906BB8F0906B80E0906BB9F0906BC4
:10093700B37452F0906AEA63A2019080A863A2019F
:100947007F061232DC021134906B6EE0C3940850BC
:100957000302113D906B7BE0FF906BB4E06F600387
:1009670002113D906B7CE0FF906BB5E06F60030276
:10097700113D906B7DE0FF906BB6E06F6003021155
:100987003D906B7EE0FF906BB7E06F600302113D17
:10099700906B7FE0FF906BB8E06F600302113D90B2
:1009A7006B80E0FF906BB9E06F600302113D906BC5
:1009B700B3E0B44415906AEAE0B4FF0E63A2019075
:1009C70080A863A2017F061232DC906EC7E0600345
:1009D7007401F0906EC87464F0906BB37452F09029
:1009E7006BB2E0646D6003020B647BFF7A1D794A8A
:1009F7001222D57BFF7A1D7964906B7BE0F52FA3DC
:100A0700E0F530A3E0F531A3E0F532A3E0F533A339
:100A1700E0F5341222D5752FFF75301D7531C1757C
:100A270032FF75331D7534CD7BFF7A1D799A1222FB
:100A3700D57BFF7A1D79D61222D57BFF7A1E793CAA
:100A47001222D57BFF7A1E7969906B81E0F52FA37F
:100A5700E0F530A3E0F531A3E0F5321222D57BFFB4
:100A67007A1E7993906B8AE0F52FA3E0F530A3E027
:100A7700F531A3E0F5321222D57BFF7A1E79C190BA
:100A87006B8EE0F52FA3E0F530A3E0F531A3E0F599
:100A9700321222D57BFF7A1E79EF906B77E0F52F24
:100AA700A3E0F530A3E0F531A3E0F5321222D57BC0
:100AB700FF7A1F7912906B73E0F52FA3E0F530A34F
:100AC700E0F531A3E0F5321222D57BFF7A1F792FAB
:100AD700906B92E0F52F1222D57BFF7A1F7959127E
:100AE70022D57BFF7A1F7982A21EE433F52F1222CB
:100AF700D57BFF7A1F79B2906EBDE0F52F1222D514
:100B07007BFF7A1F79DD906EC7E0F52F1222D57B28
:100B1700FF7A207910906AF0E0F52F1222D57BFF3B
:100B27007A20793EA211E433F52F1222D57BFF7A82
:100B370020796A906EB7E0F52FA3E0F530A3E0F5D2
:100B470031A3E0F532A3E0F533A3E0F5341222D563
:100B5700123B4B7BFF7A2079B51222D522906BB2DC
:100B6700E0644C70527E207FBB123E4E906BBAE021
:100B7700F527A3E0F528E4F5297D03AF28AE271272
:100B870040ED7E207FF6123E4EAE27AF28E4FB7D78
:100B97001012429D7E207FF9123E4E74102528F5D3
:100BA70028E43527F5270529E529C3941040CA7E8F
:100BB700207FF9123E4E22906BB2E0646C705CF5B8
:100BC7002B7E207FFB123E4EE4F52AAF2B7E007D65
:100BD700031240ED7E207FF6123E4EE4F529A82B46
:100BE700E6FF74BC2529F582E4346BF583EFF00545
:100BF7002B0529E529B410E67E6B7FBCE4FB7D104D
:100C070012429D7E207FF9123E4E052AE52AC394A3
:100C17000840B87E207FF9123E4E22906BB2E06406
:100C27004B7061F52974A42529F582E4346BF583AB
:100C3700E0603274A42529F582E4346BF583E0F48F
:100C4700602374A42529F582E4346BF583E0FF74EF
:100C5700BA2529F582E4346BF583E0B50710052939
:100C6700E529B408C090693E7432F0021134906BE4
:100C7700B27421F0301A030211347E217F36123EFE
:100C87004E021134906BB2E0B4521A201A077E213B
:100C97007F3E123E4E906BB27472F07E6B7FB27DD8
:100CA700081249D522906BB2E064497045201A07B3
:100CB7007E217F49123E4E906BBAE0F527A3E0F5FF
:100CC70028E4F529852882852783E0FF74BC252938
:100CD700F582E4346BF583EFF00528E5287002050B
:100CE700270529E529B480DC7E6B7FB27D8A12490E
:100CF700D522906BB2E064437079A3E064527046EA
:100D0700201A077E217F51123E4E906BBAE0F527DD
:100D1700A3E0F528E4F529852882852783E493FF56
:100D270074BC2529F582E4346BF583EFF00528E5DB
:100D370028700205270529E529B480DB7E6B7FB281
:100D47007D8A1249D522906BB3E064576003021184
:100D57003D906BBAE0F527A3E0F52874BC2529F58B
:100D670082E4346BAD82FC7B80AF28AE27124F45FF
:100D7700021134906BB2E064446003020E0B906B77
:100D8700BAE0FF64447003021134EFB4310CC21AA5
:100D97007E217F5A123E4E021134906BBAE0B43076
:100DA7000CD21A7E217F66123E4E021134906BBA26
:100DB700E0B4320CD21B7E217F73123E4E021134F7
:100DC700906BBAE0B4330CC21B7E217F81123E4E7A
:100DD700021134906BBAE0B4340CD21C7E217F90A0
:100DE700123E4E021134906BBAE0B4350CC21C7E31
:100DF700217F9D123E4E021134906BBAE0FF120024
:100E07001E02113490693EE07013201A077E217F7D
:100E1700AB123E4E906BB27421F002113490693ED2
:100E27007432F0906BB2E0FFB4510A908000748086
:100E3700F0C2AF80FEEF64577045201A077E217F0E
:100E4700B9123E4E906BBBE0906B6EF0E4F52990C3
:100E57006B6EE0FFE529C39F400302113474BC2584
:100E670029F582E4346BF583E0FF906BBAE025291E
:100E770024E9F582E43469F583EFF0052980D09001
:100E87006BB2E064536003020F39201A077E217F9B
:100E9700C4123E4E906B7BE0FF9069F2E06F703CAE
:100EA700906B7CE0FF9069F3E06F7030906B7DE0B2
:100EB700FF9069F4E0B50724906B7EE0FF9069F539
:100EC700E0B50718906B7FE0FF9069F6E0B5070C77
:100ED700906B80E0FF9069F7E06F6016906BB274DB
:100EE70021F0301A030211347E217FD3123E4E02C5
:100EF7001134E4F529E4F56074E92529F582E43431
:100F070069F583E0FDAF291250060529E529C39449
:100F1700FE40E29080007480F0C2AFE4907FF0F072
:100F2700A3F0907FFD74AAF0A374FFF0A37455F0AB
:100F370080FE906BB2E0644F704C906BBAE0F5277F
:100F4700A3E0F528E5284527700A201A077E217FA8
:100F5700DC123E4E201A077E217FE3123E4EE4F557
:100F67002974BC2529F582E4346BF583E085288252
:100F7700852783F00528E528700205270529E52937
:100F8700B480DE021134906BB2E0FFB44527908045
:100F9700007480F0906BBAE0FDA3E0907FF0CDF095
:100FA700A3EDF0C2AF907FFD74AAF0A374FFF0A386
:100FB7007455F080FEEF64656003021134906BBADC
:100FC700E0FFA3E0907FF0CFF0A3EFF0E4F527F583
:100FD70028D3907FF1E09528907FF0E09527402176
:100FE700E4F5602528FFE5273478FE7B80AD28AC43
:100FF70027124F4574802528F528E43527F52780E3
:10100700D07E217FE5124847EF4E60201200039003
:101017006B81EFF0120003906B82EFF012000390E8
:101027006B83EFF0120003906B84EFF07E217FEB70
:10103700124847EF4E6020120003906B8AEFF012C0
:101047000003906B8BEFF0120003906B8CEFF012A4
:101057000003906B8DEFF07E217FF1124847EF4E32
:101067006020120003906B8EEFF0120003906B8FDD
:10107700EFF0120003906B90EFF0120003906B916A
:10108700EFF07E217FF7124847EF4E6020120003F2
:10109700906B77EFF0120003906B78EFF01200037C
:1010A700906B79EFF0120003906B7AEFF07E217F5F
:1010B700FD124847EF4E6020120003906B73EFF06C
:1010C700120003906B74EFF0120003906B75EFF052
:1010D700120003906B76EFF07E227F03124847EFF2
:1010E7004E6008124CA7906B92EFF0E4F529E4F5F7
:1010F70060E52904FF74732529F582E4346BF583D1
:10110700E0FD1250060529E529C3944340E090808D
:10111700007480F0C2AFE4907FF0F0A3F0907FFD01
:1011270074AAF0A374FFF0A37455F080FE7E6B7F62
:06113700B27D081249D54B
:01113D00228F
:104F0D00AE07EEC39430400BEED394395005EE242A
:104F1D00D0FF22EEC39461400BEED394665005EEA4
:104F2D0024A9FF22EEC39441400BEED394465005C5
:084F3D00EE24C9FF22AF062299
:10519C00906AE9E004F07006906AE8E004F0906A26
:0A51AC00E8E0FEA3E0FF124E8B22A4
:1000030012519C124F0DEFC454F0FEC00612519CC6
:08001300124F0DD0E02FFF2277
:104CA700E4907003F012519C907004EFF0C39430BD
:104CB7004018E0FFD394395011907003E02441F578
:104CC70082E43469F583EFF08011907003E02441AA
:104CD700F582E43469F583E4F0800C907003E00416
:104CE700F0E0D3940840BE75320075330075340088
:0C4CF700E4F5357B017A69794112355DE6
:014D0300228D
:044847008E2C8F2DF7
:10484B00906AE8E4F0A374FFF012519CEF606EF4F1
:10485B00606B852D82852C83E493B507EC752E0157
:10486B00E52D252EF582E4352CF583E49360259018
:10487B006AE9E0252EFF906AE8E03400FE124E8BC9
:10488B00E52D252EF582E4352CF583E493B507044D
:10489B00052E80CCE52D252EF582E4352CF583E411
:1048AB009370A6E52E24FFFFE434FFFE906AE9E047
:1048BB002FF0906AE8E03EF07E007F0122E4FEFFDD
:0148CB0022CA
:103D68007E227F34124847EF4E70037F01227E2265
:103D78007F37124847EF4E600C12519CEF24D02435
:103D8800FF921E8002D21E7E227F3D124847EF4ED0
:103D9800600C12519CEF24D0906EBDF08005E49029
:103DA8006EBDF07E227F43124847EF4E600C1251E1
:103DB8009CEF24D0906EC7F08005E4906EC7F07E2B
:103DC800227F49124847EF4E600C12519CEF24D0D5
:103DD800906AF0F08005E4906AF0F07E227F4F123E
:103DE8004847EF4E600C12519CEF24D024FF9211EB
:103DF8008002C211906B7B63A201906EB763A2012F
:103E08007F061232DC30113B7E227F55124847EF85
:103E18004E6030120003906EB7EFF0120003906E00
:103E2800B8EFF0120003906EB9EFF0120003906E35
:103E3800BAEFF0120003906EBBEFF0120003906E21
:063E4800BCEFF07F002238
:10300E00C211E4906EC7F0D21EC214906EBDF09045
:10301E006AF0F0906B7B63A201906EB763A2017FA2
:10302E00061232DCE4F527E52775F003A4245BF5E0
:10303E0082E43422F583E493FB740193FA740293D1
:10304E00F912289E7003023200E4F528F529FD746A
:10305E00692DF582E43469F583E0FF70030231FBDC
:10306E00E52775F003A4245BF582E43422F583E4AE
:10307E0093FB740193FA740293F985288275830089
:10308E001228B7FEEFB5060875290105280231F79B
:10309E00E52970030231F7EE60030231F2E52724D1
:1030AE00FE60281470030231DA1470030231DE144C
:1030BE0070030231E61470030231EA240560030244
:1030CE0031FB906EC77401F00231FBD21174692D81
:1030DE00F582E43469F583E0FF642D70030231FB61
:1030EE00124F0DEFC454F0FC746A2DF582E434696E
:1030FE00F583E0FF124F0DEF2C906EB7F0746B2D31
:10310E00F582E43469F583E0FF124F0DEFC454F0FD
:10311E00FC746C2DF582E43469F583E0FF124F0DDB
:10312E00EF2C906EB8F0746D2DF582E43469F58352
:10313E00E0FF124F0DEFC454F0FC746E2DF582E4D7
:10314E003469F583E0FF124F0DEF2C906EB9F074D9
:10315E006F2DF582E43469F583E0FF124F0DEFC455
:10316E0054F0FC74702DF582E43469F583E0FF129F
:10317E004F0DEF2C906EBAF074712DF582E4346918
:10318E00F583E0FF124F0DEFC454F0FC74722DF571
:10319E0082E43469F583E0FF124F0DEF2C906EBB85
:1031AE00F074732DF582E43469F583E0FF124F0D50
:1031BE00EFC454F0FC74742DF582E43469F583E0A9
:1031CE00FF124F0DEF2C906EBCF08021D214801D9B
:1031DE00906EBD7401F08015C21E8011906AF0745D
:1031EE0001F08009E4F529F5280D02305D0527026E
:0231FE0030356A
:0132000022AB
:104DB800906DB3E0C3947C503D906DB3E0FE04F079
:104DC80074F12EF582E4346AF583EFF0BF0A279078
:104DD8006DB3E0FF04F074F12FF582E4346AF583D3
:104DE800E4F0906DB3E0FF124A57906DB37408F089
:074DF800906AF2E004F022D2
:104D5F009080007480F0906B7363A201F583F582ED
:104D6F0063A2017F081232DC906B7B63A2019080FB
:104D7F008863A2017F0A1232DC908092E4F0A37460
:104D8F0032F0A37401F0906B85E0FF9080B1F0904A
:104D9F0080E1EFF09080957455F0A3F0908000744F
:094DAF0001F09080097470F022FB
:104B5000908009E04410F09080A0E0706C9080A1FB
:104B60007482F09080A874FFF0A3F0A3F0A3F07F0C
:104B7000039080AEEFF07FCBA3EFF07F039080AC8B
:104B8000EFF0A374CBF09080007402F0906FF712F6
:104B90002A3200000000906FF7E0908040F0906FA4
:104BA000F8E0908041F0906FF9E0908042F0906FD3
:104BB000FAE0908043F0A3E4F0A3F0A3F0A3F09018
:094BC0008018F0A3F0A3F0A3F0AB
:014BC90022C9
:104C4400908009E04440F09080D17482F0906B86AB
:104C5400E0FF9080DEF0906B87E0FF9080DFF090C3
:104C640080027402F0906FFB122A32000000009060
:104C74006FFBE0908058F0906FFCE0908059F090CA
:104C84006FFDE090805AF0906FFEE090805BF0A39F
:104C9400E4F0A3F0A3F0A3F0908030F0A3F0A3F02D
:024CA400A3F07B
:014CA60022EB
:104BCA00908009E04420F09080B8E0706C9080B941
:104BDA007482F07F039080C6EFF07FCDA3EFF07F61
:104BEA00039080C4EFF0A374CDF09080C074FFF0FE
:104BFA00A3F0A3F0A3F09080017402F0906FFF126B
:104C0A002A3200000000906FFBE090804CF0906F19
:104C1A00FCE090804DF0906FFDE090804EF0906F38
:104C2A00FEE090804FF0A3E4F0A3F0A3F0A3F0908D
:094C3A008024F0A3F0A3F0A3F024
:014C4300224E
:104951008C278D28A907EAFDE975F018A424ACFF7E
:10496100E5F034808F82F583EDF0EBFDE975F01809
:10497100A4FFAEF024ACFBEE34808B82F583A3ED73
:10498100F08528828C83E0FDEF24A8FFEE3480FEC1
:104991008F82F583EDF08528828C83A3E08F828E50
:1049A10083A3F0852882852783A3A3E0FDE975F021
:1049B10018A424A8FFE5F03480FE8F82F583A3A319
:1049C100EDF08528828C83A3A3A3E08F828E83A33D
:0449D100A3A3F0228A
:0649D5008D2CAB07AA06C1
:1049DB00906FF7E0FCA3E0FDA3E0FEA3E0F5308EC3
:1049EB002F8D2E8C2DAE02AF038E838F8263A2018F
:1049FB00E52F540744C0F58385308263A201AF2CA9
:104A0B00123345908000E020E5F9E4FCFDFEE53033
:104A1B00252CF530EE352FF52FED352EF52EEC350B
:104A2B002DF52D908040E52DF0A3E52EF0A3E52F7D
:104A3B00F0A3E530F09080007420F0AF30AE2FADD6
:0B4A4B002EAC2D906FF7122A26AF2C26
:014A5600223D
:064AD5008D27AB07AA06C5
:104ADB00906FFBE0FCA3E0FDA3E0FEA3E0F52B8EC3
:104AEB002A8D298C28AE02AF038E838F8263A2019D
:104AFB00E52A540744D0F583852B8263A201AF27A7
:104B0B00123345E4FCFDFEE52B2527F52BEE352A6C
:104B1B00F52AED3529F529EC3528F528908058E54F
:104B2B0028F0A3E529F0A3E52AF0A3E52BF090806C
:104B3B00027420F0AF2BAE2AAD29AC28906FFB127C
:044B4B002A26AF2740
:014B4F002243
:024423008F28E0
:10442500908001E030E5037F0022906FFFE0FCA360
:10443500E0FDA3E0FEA3E0F52C8E2B8D2A8C2990C0
:104445006EB763A201E52B540744C8F583852C821A
:1044550063A2017F0612335BE52C2406F52CE435B7
:104465002BF52BE4352AF52AE43529F529906DB588
:1044750063A201E52B540744C8F583852C8263A20A
:1044850001AF2812335BE4FCFDFEE52C2528F52C55
:10449500EE352BF52BED352AF52AEC3529F5299046
:1044A500804CE529F0A3E52AF0A3E52BF0A3E52C44
:1044B500F09080017420F0AF2CAE2BAD2AAC299082
:0744C5006FFF122A26AF2849
:0144CC0022CD
:103C64009081E0E0F5270527052705270527052787
:103C740005270527052705270527908010E0F52A45
:103C8400A3E0F52BA3E0F52CA3E0F52D9081E1E072
:103C9400F5270527052705270527052705270527D0
:103CA400052705270527908014E0F52EA3E0F52FBE
:103CB400A3E0F530A3E0F531E530B52C08E531B5E6
:103CC4002D037F0022E4F527E530540744E0F58313
:103CD40085318263A201906BB263A2017F08123323
:103CE40073906BB463A201906AEA63A2017F061227
:103CF40032DC906BB2E0F528A3E0F529E4F52790D7
:103D04006BB2E0702AA3E024F8F527E530540744A9
:103D1400E0F58385318274082582F582E43583F5E4
:103D24008363A201906BB263A201AF27123373AE17
:103D340028E4FCFDE5312529F531E5303EF530ED8B
:103D4400352FF52FEC352EF52E908014E52EF0A3AB
:103D5400E52FF0A3E530F0A3E531F0908000744046
:033D6400F0AF2796
:013D67002239
:103701009081E6E0F52705270527052705270527E9
:1037110005270527052705270527908028E0F52A95
:10372100A3E0F52BA3E0F52CA3E0F52D9081E7E0D4
:10373100F527052705270527052705270527052738
:1037410005270527052790802CE0F52EA3E0F52F0E
:10375100A3E0F530A3E0F531E4F527E530B52C0A17
:10376100E531B52D05C21802385BE530540744F048
:10377100F58385318263A201906BB263A2017F0858
:10378100123373906BB2E0F528A3E0F529E52945E2
:103791002870099080027410F07F0022906EBEE0C4
:1037A100FFF4602D906BB4E06F7076906EBFE0FF18
:1037B100906BB5E06F706A906EC0E0FF906BB6E001
:1037C1006F705E906EC1E0FF906BB7E06F6022801A
:1037D10050906BB4E0906EBEF0906BB5E0906EBF10
:1037E100F0906BB6E0906EC0F0906BB7E0906EC158
:1037F100F0906BB2E0702AA3E024F8F527E530548D
:103801000744F0F58385318274082582F582E43519
:1038110083F58363A201906BB263A201AF271233D8
:1038210073AE28E4FCFDE5312529F531E5303EF59F
:1038310030ED352FF52FEC352EF52EAF2DAE2CAD0D
:103841002BAC2AAB31AA30A92FA82ED3122A1540AE
:10385100099080027410F07F002290802CE52EF0F8
:10386100A3E52FF0A3E530F0A3E531F090800274D9
:0438710040F0AF274D
:013875002230
:1039E5009081E3E0F5270527052705270527052706
:1039F5000527052705270527052790801CE0F52ABB
:103A0500A3E0F52BA3E0F52CA3E0F52D9081E4E0F0
:103A1500F527052705270527052705270527052751
:103A2500052705270527908020E0F52EA3E0F52F33
:103A3500A3E0F530A3E0F531E4F527E530B52C0A30
:103A4500E531B52D05C219023B30E530540744E890
:103A5500F58385318263A20190683E63A2017F0EE2
:103A650012338990683EE0F528A3E0F52990684671
:103A7500E0FFF46045906EB7E0FEEF6E706EA3E078
:103A8500FF906847E06F7064906EB9E0FF906848FA
:103A9500E06F7058906EBAE0FF906849E06F704C27
:103AA500906EBBE0FF90684AE06F7040906EBCE09E
:103AB500FF90684BE06F60048032D2D990683EE099
:103AC500702AA3E024F2F527E530540744E8F5838E
:103AD500853182740E2582F582E43583F58363A2F0
:103AE5000190683E63A201AF27123389AE28E4FC3A
:103AF500FDE5312529F531E5303EF530ED352FF57C
:103B05002FEC352EF52EAF2DAE2CAD2BAC2AAB31CF
:103B1500AA30A92FA82ED3122A155006E529452823
:103B250070099080017410F07F0022908020E52EAE
:103B3500F0A3E52FF0A3E530F0A3E531F090800187
:053B45007440F0AF2701
:013B4A002258
:043E4E008E2D8F2EF8
:103E5200906FF7E0FCA3E0FDA3E0FEA3E0F5348E53
:103E6200338D328C31E534FFE5335407FEE42FF510
:103E720030EE34C0F52F853082F5837423F005309F
:103E8200E5307002052F532FC7F582852F83740A00
:103E9200F00530E5307002052F532FC7906B7B631E
:103EA200A201852F8385308263A2017F06123345EA
:103EB20074062530F530E4352FF52F852D83852EB8
:103EC2008263A201852F8385308263A20112332986
:103ED200908000E020E5F9E4FCFDFE906FF7E0F849
:103EE200A3E0F9A3E0FAA3E02FFFEE3AFEED39FDDD
:103EF200EC38FCEF2408FFE43EFEE43DFDE43CFC2C
:103F0200906FF7122A26906FF7E0908040F0906F42
:103F1200F8E0908041F0906FF9E0908042F0906F6D
:0C3F2200FAE0908043F09080007420F0E2
:013F2E002270
:06429D008E2D8F2E8D2FE7
:1042A300906FF7E0FCA3E0FDA3E0FEA3E0F5358EFD
:1042B300348D338C32E535FFE5345407FEE42FF5B6
:1042C30031EE34C0F530853182F5837423F0053146
:1042D300E531700205305330C7F582853083EBF04A
:1042E3000531E531700205305330C7906B7B63A213
:1042F3000185308385318263A2017F0612334574C1
:10430300062531F531E43530F530852D83852E8250
:1043130063A20185308385318263A201AF2F1233FB
:1043230045908000E020E5F97408252FF52FFFE480
:10433300FCFDFEE5352FF535EE3534F534ED35333B
:10434300F533EC3532F532908040E532F0A3E533B6
:10435300F0A3E534F0A3E535F09080007420F0AFCE
:0D43630035AE34AD33AC32906FF7122A2620
:01437000222A
:024A57008F408E
:104A5900906FF7E0FCA3E0FDA3E0FEA3E0F5448E30
:104A6900438D428C41E544FFE5435407FEE42FFFA3
:104A7900EE34C0906AF163A201F5838F8263A201CB
:104A8900AF40123345908000E020E5F9E4FCFDFEDB
:104A9900E5442540F544EE3543F543ED3542F5420D
:104AA900EC3541F541908040E541F0A3E542F0A3A2
:104AB900E543F0A3E544F09080007420F0AF44AEE4
:0B4AC90043AD42AC41906FF7122A266B
:014AD40022BF
:0640ED008E2C8F2DAB05A7
:1040F300906FF7E0FCA3E0FDA3E0FEA3E0F5338EB1
:10410300328D318C30E533FFE5325407FEE42FF571
:104113002FEE34C0F52E852F82F5837423F0052FFF
:10412300E52F7002052E532EC7F582852E83EBF003
:10413300052FE52F7002052E906B7B63A201852E60
:1041430083852F8263A2017F061233457406252FD0
:10415300F52FE4352EF52E532EC7E52C852F8285BA
:104163002E83F0052FE52F7002052E532EC7F582FF
:10417300852E83E52DF0052FE52F7002052E532E96
:10418300C7908000E020E5F9E533240AF533E435F0
:1041930032F532E43531F531E43530F53090804095
:1041A300E530F0A3E531F0A3E532F0A3E533F09079
:1041B30080007420F0AF33AE32AD31AC30906FF786
:0341C300122A2697
:0141C60022D6
:10456900E4F527E5272401FFE433FE124E8B74732B
:104579002527F582E4346BF583EFF00527E527C39A
:10458900943F40DFE4F527E527247FFFE433FE125B
:104599004E8B74692527F582E43469F583EFF0744D
:1045A900692527F582E43469F583E0FF6003B4FFE8
:1045B9001D74692527F582E43469F5837420F07444
:1045C9006A2527F582E43469F583E4F08009052733
:1045D900E527C3948040B0E49069E8F0F527AF2758
:1045E9007E00124E8B74E92527F582E43469F58340
:0B45F900EFF00527E527C394FE40E328
:014604002293
:10515F00E4FDFCC3ED9FEC9E5015E4FBFA0BBB0086
:0F516F00010ABA01F8BB90F50DBD00010C80E4F8
:01517E00220E
:0D5227004390014390025390FE5390FD22EE
:0D5234005390FD5390FE43900243900122E1
:0E5209005390FD439002E5905408FF5390FD32
:015217002274
:0D5241005390FD4390014390025390FD22D5
:07526A00AE071FEE70FA22EF
:024FDA00AD0721
:104FDC00E4FC5390FDEDA804088002C333D8FC30E8
:104FEC00E70543900180035390FE7F0512526A43FC
:094FFC0090020CBC08DC5390FD8E
:015005002288
:10505A00E4FF5390FD7E07439002E59030E00D7423
:10506A0001A806088002C333D8FC42075390FD1EEC
:08507A00C3EE6480948050DF56
:01508200220B
:10500600AB05AA071252277FA0124FDA125209AF38
:1050160002124FDA125209AF03124FDA1252091274
:0A50260052347F0A7E0012515F220F
:044E8B00AB07AA06C1
:104E8F00C3EB94FFEA9400400DE42BF58274773A5C
:104E9F00F583E493FF221252277FA0124FDA1252AA
:104EAF0009AF03124FDA1252091252277FA1124F84
:0D4EBF00DA12520912505A125241125234A6
:014ECC0022C3
:024F45008B2CB3
:104F4700A2AF921FC2AF85A22D53A2FE8E838F827E
:104F570005A28C838D8274091233A1E52C53A2FE1E
:104F670043A2201233A353A2DF852DA2A21F92AF23
:014F7700FF3A
:014F78002216
:10517F00A2AF921FC2AF8C838D82EF1233A143A2D5
:0C518F00201233A353A2DFA21F92AFFF37
:01519B0022F1
:0250D2008F2726
:1050D400A2AF921FC2AFE4F5838D8274061233A18E
:1050E400E52743A2201233A353A2DFA21F92AF7F6E
:0150F40001BA
:0150F5002298
:0250F6008F2702
:1050F800A2AF921FC2AFE4F5838D82740A1233A166
:10510800E52743A2201233A353A2DFA21F92AF7F49
:015118000195
:015119002273
:10320100A907E7FFA805EF93C3966008403B74FC4C
:103211002FFF80F00F08EF93C3966008402B74FBDB
:103221002FFF80E00F08EF93C3966008401B74FAEC
:103231002FFF80D00F08EF93D3966008400B74F9ED
:103241002FFF80C01F1F1F1F1FEF54FEF80303F73E
:10325100E893FC08E893FD08E893FE08E893FF2251
:1032610009E993C39D6008402974FB29F980F1099C
:10327100E993C39E6008401A74FA29F980E209E9CA
:1032810093D39F6008400B74F929F980D319191958
:103291001919E9C313C313FF22740093F8ECC398FF
:1032A1004024701F740193F8EDC398401970147491
:0E32B1000293F8EEC398400E7009740393F870
:1032BF00EFC39840037F00227F0122EDF8E6F0086C
:1032CF00A3DFFA22EDF8E0F608A3DFFA22E0A3630A
:1032DF00A201F0A363A201DFF475A20022E0A363B1
:1032EF00A201F0A363A201E0A363A201F0A363A272
:1032FF0001E463A201F0A363A201DFE175A2002242
:10330F00E0A363A2016DFE936CFDEE058393FC15A4
:10331F008363A201DFEA75A200227F00E493A36317
:10332F00A201F00F600CA3E583C2E3F58363A20152
:10333F0080EA75A20022E0A363A201F0A3E583C295
:10334F00E3F58363A201DFEE75A20022E0A363A27F
:10335F0001F0A3E583C2E4D2E3F58363A201DFECBE
:10336F0075A20022E583C2E3F583E0A363A201F017
:10337F00A363A201DFEE75A20022E583C2E4D2E3CC
:10338F00F583E0A363A201F0A363A201DFEC75A2B2
:10339F000022F922C002C004C00612FFF0D006D0EE
:0433AF0004D0022222
:10472D000A536572763A004572724C656E210A0025
:10473D00205544502054696D654750530A00200A96
:10474D00444154414752414D3A20002043414E20AF
:10475D0054696D654750530A002054726173735349
:10476D00656E644552520A000ACEF8C4EBE8EDFBC3
:10477D0043414E210A000A45727241647243414E13
:10478D003A000A00205265496E69742043414E0A71
:10479D00002043414E283029203E20544F210A004D
:0E47AD0020545520300A0020545520310A00B7
:03001E00E4FF22DA
:10508300C2A9438902758C48758A4875D90475DBB2
:105093004875DC4875DD4875DE48E4F5E9F5F9D275
:0850A300D9C2DAD28CD2DE2260
:104FAC00C2D9906EDDE07013E5E92419F5EB30D72A
:104FBC0006E5F904F5FB2285F9FB22E5E924C8F5A1
:0E4FCC00EB30D706E5F904F5FB2285F9FB2250
:104DFF00C2D9906EDDE0702C302C16E5E92432F527
:104E0F00EB30D707E5F904F5FB800385F9FBC22CDE
:104E1F0022E5E92405F5EB30D706E5F904F5FB2289
:104E2F0085F9FB22E5E92432F5EB30D706E5F904E5
:074E3F00F5FB2285F9FB22BF
:1050AB00125083906EDDE0C3946450061241C71218
:1050BB004FAC12527ED22BE4F556906FF5F0F545BE
:0750CB00F55AC22CF5582232
:104E4600EF24FCF545201A127E477F2D123E4E7E3A
:104E56006B7FB6E4FBAD4512429DE545D3940D400C
:104E660010201A077E477F34123E4EE4F545D229BC
:104E760022906BB663A201906FE563A201AF451263
:054E860032DCC229220C
:0F521800D3EF6480948D5006E55A70028F5A22AE
:1025CF0020D9030226AC202B030226ACE55A605219
:1025DF0090683E540FFF7D471232D3E54764017078
:1025EF001E906846E0B4FF0ED22D201A127E477F50
:1025FF003D123E4E8009302D06E4F55A0226AC12EC
:10260F004FAC123F2F201A077E477F4B123E4E20B2
:10261F001A0B7E687F3EE4FBAD5A12429DE4F55AD9
:10262F00807BE5456043906FE9E02405F527D3945F
:10263F000D4007E4F545D2298063906FE5E52754F7
:10264F000FFF7D471232D3E54730E702D22CE54723
:10265F00B40109302D06E54A64016003123F2F12C1
:10266F004FACE4F545D2298034E557601E906EC912
:10267F00540FFF7D471232D3E547B40103202D03DA
:10268F00123F2F124FACE4F557801220010C906EC1
:10269F00DDE0C3946450031248CC124FAC124605D0
:1026AF008F27EF700302277D124DFFE4F558E547A2
:1026BF00547EB54703124D04E547B4010CD22D20CB
:1026CF001A077E477F58123E4EE559C394C8502DC6
:1026DF0030132AE547B4420DE54AB40208906AF078
:1026EF00E06401601874DE2559F582E4346EF583D9
:1026FF00E5272559F5597D47AF271232CA301121E9
:10270F00E54720E71C906DB57D47AF271232CAAF62
:10271F0027124423EF700A201A077E477F66123E66
:10272F004EE54754817047E527D3940D400C201A8E
:10273F003D7E477F75123E4E8034E549D394074066
:10274F0028201A2A7E477F83123E4E9069417D478B
:10275F00AF271232CA7E697F41E4FBAD2712429D3B
:10276F007E477F8F123E4E8005AF27122B64301DA0
:10277F002030101B906EDDE0C3946450120558E5B5
:10278F005894F0400A9080007480F0C2AF80FEC26F
:10279F001D201203022898E5566031D3940140049E
:1027AF0015568028906FF5E004F0E0D39403400DA8
:1027BF00201A077E477F91123E4E1250AB201A0708
:1027CF007E477F9E123E4EE4F556D22B302A43E5CC
:1027DF0057703F906EC904F0A37408F0A37480F093
:1027EF00A37401F0A37406F0906FE0E0906ECEF04A
:1027FF00906FE1E0906ECFF0906FE2E0906ED0F0CE
:10280F00906FE3E0906ED1F0E4A3F0A3F075570B57
:10281F00C22A302872906FDEE07035E55770319024
:10282F006EC97442F0A37408F0906FDFE0906ECB26
:10283F00F0906FE4E0906ECCF0A37401F075570642
:10284F00201A077E477FAD123E4E906FDEE004F0F8
:10285F00906FDEE06402702FE557702B906EC97495
:10286F0002F0A37408F0906FDFE0906ECBF0A3F04E
:10287F00A37401F0755706201A077E477FB4123EE6
:0E288F004E906FDEE004F0C212120026C2105E
:01289D002218
:104F7900E559602CE4906CB2F0A3E559F0906EB657
:104F8900E0906CB4F0A37419F0906EDE63A2019006
:104F99006CB663A201AF591232DCE4F5597F0122E4
:034FA9007F002264
:0B524E00302905C2297F01227F0022C9
:0100210022BC
:06527800E4F559F54522A2
:0A525900E4906941F0A3F0A3F022F5
:0752710020457272210A00C2
:1051B600EF600A7B10E4FD7F0C125030227B107DDD
:0751C600107F0C1250302293
:1041C700D29475C353C29475C5C0E5C4B480FB854A
:1041D700C528D2947DE07F0F12513E906EDDE044FA
:1041E70080FD7F2A12513E7D247F2912513E7D0496
:1041F7007F2812513EE4FD7F2B12513E752A20E4A1
:10420700F529E4FDAF2A12513E052A0529E529C300
:10421700940840EEE4F52AF529E4FDAF2A12513E51
:10422700052A0529E529C3940C40EE7D087F051270
:10423700513E752A10E4F529E4FDAF2A12513E05D7
:104247002A0529E529C3940C40EE7D3C7F0C1251C9
:104257003E7D077F0F12513E7DFF7F2B12513E752A
:104267002A30E4F528E4F529E4FDAF2A12513E058A
:104277002A0529E529C3940E40EE052A052A0528B3
:10428700E528C3940340DE7D047F6012513EE4FDC0
:054297007F7012513E92
:01429C0022FF
:10511A00C29475C503E5C4B480FBAEC58FC5E5C4AA
:10512A00B480FBAEC5E4F5C5E5C4B480FBAEC5D218
:03513A0094AF0629
:01513D00224F
:10513E00C29475C502E5C4B480FBAEC58FC5E5C487
:10514E00B480FBAEC58DC5E5C4B480FBAEC5D294AC
:01515E00222E
:10503000C29475C505E5C4B480FBAEC58FC5E5C493
:10504000B480FBAEC58BC5E5C4B480FBAEC58DC5D1
:09505000E5C4B480FBAEC5D294A6
:015059002234
:10400F00C29475C503E5C4B480FBAEC5EF60047EF2
:10401F007080027E608EC5E5C4B480FBAEC5E4F54A
:10402F00C5E5C4B480FB85C546E4F5C5E5C4B480D9
:10403F00FB85C547E4F5C5E5C4B480FB85C548E4F9
:10404F00F5C5E5C4B480FB85C549E4F5C5E5C4B441
:10405F0080FB85C54AE4F5C5E5C4B480FB85C54B37
:10406F00E54B540FFE60741EE4F5C5E5C4B480FB48
:10407F0085C54CEE60651EE4F5C5E5C4B480FB85CF
:10408F00C54DEE60561EE4F5C5E5C4B480FB85C58D
:10409F004EEE60471EE4F5C5E5C4B480FB85C54F01
:1040AF00EE60381EE4F5C5E5C4B480FB85C550EE5F
:1040BF0060291EE4F5C5E5C4B480FB85C551EE60EB
:1040CF001A1EE4F5C5E5C4B480FB85C552EE600B3E
:0D40DF00E4F5C5E5C4B480FB85C553D2945B
:0140EC0022B1
:103F2F00906EDDE0C39464400302400CC29475C5EB
:103F3F0002E5C4B480FBAFC575C531E5C4B480FBE1
:103F4F00AFC5E54B540FFE8547C5E5C4B480FBAF45
:103F5F00C58548C5E5C4B480FBAFC58549C5E5C473
:103F6F00B480FBAFC5854AC5E5C4B480FBAFC5853A
:103F7F004BC5E5C4B480FBAFC5EE606C1E854CC568
:103F8F00E5C4B480FBAFC5EE605E1E854DC5E5C4CC
:103F9F00B480FBAFC5EE60501E854EC5E5C4B4803E
:103FAF00FBAFC5EE60421E854FC5E5C4B480FBAFC5
:103FBF00C5EE60341E8550C5E5C4B480FBAFC5EEB9
:103FCF0060261E8551C5E5C4B480FBAFC5EE6018F1
:103FDF001E8552C5E5C4B480FBAFC5EE600A85539C
:103FEF00C5E5C4B480FBAFC5D2947F02C29475C53A
:0F3FFF0081E5C4B480FBAFC5D29475560AC22BBE
:01400E00228F
:104D0400C29475C502E5C4B480FBAFC575C541E561
:104D1400C4B480FBAFC58547C5E5C4B480FBAFC54B
:104D24008548C5E5C4B480FBAFC58549C5E5C4B4B1
:104D340080FBAFC5854AC5E5C4B480FBAFC5E4F5C7
:104D4400C5E5C4B480FBAFC5D2947F02C29475C5D7
:0A4D540082E5C4B480FBAFC5D29421
:014D5E002232
:1048CC00C29475C502E5C4B480FBAFC575C551E58E
:1048DC00C4B480FBAFC574872513F582E43461F54D
:1048EC0083E0F5C5E5C4B480FBAFC575C508E5C468
:1048FC00B480FBAFC574882513F582E43461F5836D
:10490C00E0F5C5E5C4B480FBAFC575C50FE5C4B40F
:10491C0080FBAFC50513051374872513F582E434AA
:10492C0061F583E07002F513E4F5C5E5C4B480FBD2
:10493C00AFC5D2947F02C29475C584E5C4B480FB24
:04494C00AFC5D2948D
:014950002244
:104605003092037F00227F2C12511A8F28E5283023
:10461500E209D22BE4F556906FF5F0E52830E55820
:10462500201A077E527F71123E4E7F2D12511A8F2E
:1046350029201A11E528FE7C00E42529FFEC3EFE21
:104645007D031240EDE4FBAD297F2D125030201A79
:104655001BE52830E016E4FF12400FE547FE7C001D
:10466500E4254BFFEC3EFE7D031240EDAB28E4FD57
:104675007F2C1250307F0022E4F529E52830E00D2B
:10468500E4FF12400FE54B54072405F529AB28E458
:08469500FD7F2C125030AF290B
:01469D0022FA
:10113E005452414E5A004D415842005254530044AD
:10114E00454C4159004D4F4445004B5000545500FD
:10115E0043414E004B565400415400444952004303
:10116E00414E4D4F4E00475254494D45005449543F
:10117E0053005453494E5600003E2A2C312CCFE0DA
:10118E00F0E0ECE5F2F0FB20F3EFF0E0E2EBFFFE37
:10119E00F9E5E3EE20EAEEEDF2F0EEEBEBE5F0E052
:1011AE0020CACF20C8F1E5F2FC0A003E4C2C6B3071
:1011BE00312C25732C43EAEEF0EEF1F2FC20EDE03B
:1011CE0020F8E8EDE52043414E2C30202D2035301F
:1011DE0030EAE1283530EC292C31202D203530EA4B
:1011EE00E128353030EC290A0030202D2035303002
:1011FE00EAE1283530EC290031202D203530EAE1A6
:10120E0028353030EC29003E532C6B30322C2562C1
:10121E00752CCCE0EAF12E20E0E4F0E5F120E1EBD4
:10122E00EEEAE020D2D128302D38290A003E532C88
:10123E006B30332C2562752CCCE0EAF12E20E0E4E5
:10124E00F0E5F120E1EBEEEAE020D2C8D228302D15
:10125E0038290A003E532C6B30342C2562752CCC69
:10126E00E0EAF12E20E0E4F0E5F120E1EBEEEAE039
:10127E0020D2D328302D38290A003E422C6330313B
:10128E002C2562752CC2F2EEF0E8F7EDFBE920EAB0
:10129E00EEEDF2F0EEEBEBE5F020EDE020F8E8ED10
:1012AE00E50A003E2A2C312CCFE0F0E0ECE5F2F01E
:1012BE00FB20EFF0EEF2EEEAEEEBE020C3F0E0ED15
:1012CE00E8F220EFEE20EFEEF0F2F320525332333D
:1012DE00320A003E432C61636B2C25732CCFEEF04B
:1012EE00FFE4EEEA20C0D4C10A00312DD2D128305D
:1012FE002B312920322DD2C8D228302920332DD29D
:10130E00D320342DD2C8D228312920352DD2D12840
:10131E00322B332920382DD2C8C8003E4C2C6B30CE
:10132E00352C256C752CD1EAEEF0EEF1F2FC20EEA8
:10133E00E1ECE5EDE020EDE020EFEEF0F2F32C3104
:10134E0030302C3230302C3330302C3630302C3193
:10135E003230302C323430302C343830302C393668
:10136E0030302C31393230302C33383430302C355B
:10137E00373630302C3131353230300A003E532C76
:10138E006B30362C2562752CCDEEECE5F020CACFF5
:10139E00200A003E422C6730312C2562752CCCE0A1
:1013AE00E3E8F1F2F0E0EBFC0A003E422C6730324B
:1013BE002C2562752CC8EDE2E5F0F2E8F0EEE2E0E5
:1013CE00F2FC20E7EDE0F7E5EDE8FF20D2D10A00D0
:1013DE003E422C6730332C2562752CC7E0EFF0E0CF
:1013EE00F8E8E2E0F2FC20E2F0E5ECFF20F1E5F0B7
:1013FE00E2E5F0E00A003E422C6730342C2562759F
:10140E002CC2FBF1F2E0E2EBFFF2FC20525453202F
:10141E00EFF0E820EFE5F0E5E4E0F7E50A003E53F3
:10142E002C6730352C2562752CC7E0E4E5F0E6EA32
:10143E00E020EFE5F0E5E4E0F7E820EFEEF1EBE594
:10144E002052545320282A3130ECF1290A003C2135
:10145E00003C6B30313D003C6B30323D003C6B301C
:10146E00333D003C6B30343D003C6330313D003C3D
:10147E006B30353D003C6B30363D003C6730313DC6
:10148E00003C6730323D003C6730333D003C6730F6
:10149E00343D003C6730353D000ACFE5F0E5E4E031
:1014AE00F7E03A2000544949204379636C650A00FD
:1014BE005453204379636C650A0054530A0054490F
:1014CE00540A005455204F4B0A005455204469616C
:1014DE00670A005455205265710A00205455205455
:1014EE00696D654F5554210A000ACFF0E8E5EC3AD4
:1014FE0020000A4352432045525221000AD7F3E6F8
:10150E00EEE920EDEEECE5F020CACF21000A52659F
:10151E007154533120000A52657154533520000A1C
:10152E0052657154495420000ACFF0E8EDFFF2E005
:10153E0020EAEEECE0EDE4E020D2D320002020D231
:10154E00D320E7E0EDFFF2EE210A000ACDE520EF11
:10155E00EEEDFFEB20F2E8EF20EFE0EAE5F2E0211E
:10156E000A0000112332465765748C9DAFBECADB4C
:10157E00E9F810013322564775649C8DBFAEDACB65
:10158E00F9E82130021367764455ADBC8E9FEBFA15
:10159E00C8D93120120377665445BDAC9E8FFBEA45
:1015AE00D8C94253617004152736CEDFEDFC8899F9
:1015BE00ABBA5243716014053726DECFFDEC988925
:1015CE00BBAA6372405125340617EFFECCDDA9B8D5
:1015DE008A9B7362504135241607FFEEDCCDB9A805
:1015EE009A8B8495A7B6C2D3E1F008192B3A4E5FB9
:1015FE006D7C9485B7A6D2C3F1E018093B2A5E4FE5
:10160E007D6CA5B48697E3F2C0D129380A1B6F7E94
:10161E004C5DB5A49687F3E2D0C139281A0B7F6EC4
:10162E005C4DC6D7E5F48091A3B24A5B69780C1D78
:10163E002F3ED6C7F5E49081B3A25A4B79681C0DA4
:10164E003F2EE7F6C4D5A1B082936B7A48592D3C54
:10165E000E1FF7E6D4C5B1A092837B6A58493D2C84
:10166E001E0F0089129B24AD36BF48C15AD36CE5BC
:10167E007EF78108931AA52CB73EC940DB52ED6464
:10168E00FF76028B109926AF34BD4AC358D16EE750
:10169E007CF5830A9118A72EB53CCB42D950EF6644
:1016AE00FD74048D169F20A932BB4CC55ED768E130
:1016BE007AF3850C971EA128B33ACD44DF56E96024
:1016CE00FB72068F149D22AB30B94EC75CD56AE310
:1016DE0078F1870E951CA32AB138CF46DD54EB6204
:1016EE00F97008811A932CA53EB740C952DB64ED00
:1016FE0076FF89009B12AD24BF36C148D35AE56CE4
:10170E00F77E0A8318912EA73CB542CB50D966EFCF
:10171E0074FD8B029910AF26BD34C34AD158E76EC3
:10172E00F57C0C851E9728A13AB344CD56DF60E9AF
:10173E0072FB8D049F16A920BB32C54CD75EE168A3
:10174E00F37A0E871C952AA338B146CF54DD62EB8F
:10175E0070F98F069D14AB22B930C74ED55CE36A83
:10176E00F1780008040C020A060E0109050D030BA0
:10177E00070FFF113EFF1144FF1149FF114DFF11DD
:10178E0053FF1158FF115BFF115EFF1162FF1166CF
:10179E00FF1169FF116DFF1174FF117BFF1180FFA7
:0217AE001186A2
:1051E100EF540F90177093FEC454F0FEEFC4540FA8
:0451F100932EFF22D8
:0300230002469EF4
:0B469E00C0E0C083C082C0D075D018FF
:1046A90030984EC298755E01AF99200644200209E0
:1046B900EF6402703CD2028038300A04C20A8022B8
:1046C900BF0904D20A802ABF0205530B808022BF8A
:1046D9000310906614E50BF0630B80530B80C20244
:1046E900800F7437250BF582E43466F583EFF00506
:1046F9000B309927300322906185E0FFE50CC39FB9
:104709004006C203D20D8011AF0C050C74372FF58A
:0B47190082E43467F583E0F599C29953
:09472400D0D0D082D083D0E03265
:103B4B007BFF7A1179871222D5906EDDE0701475A8
:103B5B002FFF7530117531F77BFF7A1179B912226E
:103B6B00D58012752FFF7530127531067BFF7A11D8
:103B7B0079B91222D57BFF7A127915906186E0F51F
:103B8B002F1222D57BFF7A12793B906101E0F52F42
:103B9B001222D57BFF7A127962906100E0F52F1229
:103BAB0022D57BFF7A127988A201E433F52F1222FA
:103BBB00D57BFF7A1279B11222D5752FFF75301292
:103BCB007531F87BFF7A1279E11222D5906838E0D3
:103BDB00FEA3E0FFC3E49FFFE49EFEAB07FA339521
:103BEB00E0F9F87F007E8C7D0A7C001229758F32FC
:103BFB008E318D308C2F7BFF7A1379291222D57B56
:103C0B00FF7A13798B906403E0F52F1222D57BFF9B
:103C1B007A1379A1A20EE4336401F52F1222D57B1E
:103C2B00FF7A1379B8A209E433F52F1222D57BFF63
:103C3B007A1379DEA204E433F52F1222D57BFF7AB7
:103C4B00147904A20BE433F52F1222D57BFF7A14DF
:093C5B00792C85092F1222D522D3
:103876007E147F5C124847EF4E70037F0122E4906E
:103886006EDDF07E147F5F124847EF4E60151251D1
:103896009CBF3106906EDD740AF0BF3206906EDD75
:1038A6007464F07E147F65124847EF4E600A124C2E
:1038B600A7906186EFF080069061867402F07E1410
:1038C6007F6B124847EF4E600A124CA7906101EFDA
:1038D600F080069061017402F07E147F71124847F1
:1038E600EF4E600A124CA7906100EFF080069061DF
:1038F600007402F07E147F77124847EF4E600D1277
:103906004CA7EC4D4E4F24FF92018002C2017E145B
:103916007F7D124847EF4E6023124CA7A804A905E5
:10392600AA06AB077F007E8C7D0A7C0012297512E1
:103936002A07906838EEF0A3EFF0800A9068387492
:10394600FFF0A374DCF07E147F83124847EF4E60CD
:103956000A124CA7906403EFF0800690640374018A
:10396600F07E147F89124847EF4E600E12519CEF8D
:1039760024D0640124FF920E8002C20E7E147F8F33
:10398600124847EF4E600C12519CEF24D024FF9250
:10399600098002C2097E147F95124847EF4E600CDB
:1039A60012519CEF24D024FF92048002C2047E149C
:1039B6007F9B124847EF4E600C12519CEF24D02497
:1039C600FF920B8002C20B7E147FA1124847EF4E76
:0E39D6006007124CA78F098003E4F5097F00FB
:0139E40022C0
:102E0500E4F527E52775F003A42480F582E434175B
:102E1500F583E493FB740193FA740293F912289EE7
:102E2500700302300DE4F529F52AF5287469252883
:102E3500F582E43469F583E0FF7003023008E52785
:102E450075F003A42480F582E43417F583E493FB3D
:102E5500740193FA740293F9852982758300122807
:102E6500B7FEEFB50608752A010529023003E52AE4
:102E75007003023003EE6003022FFEE527B40F0056
:102E85004003023008902E91F8282873022EBE02C6
:102E95002F05022F3E022F43023008022F9B0230DE
:102EA50008022F6E023008023008022FC8022FF2E6
:102EB500022FF6023008022FFA74692528F9E43446
:102EC50069FA7B01C0031B8B32753300753400E44E
:102ED500F535D00312355D8F2E8E2D8D2C8C2BABB9
:102EE5002EAA2DA92CA82B7F007E8C7D0A7C001292
:102EF5002975122A07906838EEF0A3EFF002300822
:102F050074692528F582E43469F583E024D090615D
:102F150086F0746A2528F582E43469F583E024D0C7
:102F2500906101F0746B2528F582E43469F583E03E
:102F350024D0906100F0023008D20B023008746989
:102F45002528F9E43469FA7B01C0031B8B327533FC
:102F550000753400E4F535D00312355D8F2E8E2DC6
:102F65008D2C8C2B8F0902300874692528F9E434DF
:102F750069FA7B01C0031B8B32753300753400E49D
:102F8500F535D00312355D8F2E8E2D8D2C8C2B9023
:102F95006EDDEFF0806D74692528F9E43469FA7BFC
:102FA50001C0031B8B32753300753400E4F535D051
:102FB5000312355D8F2E8E2D8D2C8C2B906403EF97
:102FC500F0804074692528F9E43469FA7B01C0036F
:102FD5001B8B32753300753400E4F535D00312359B
:102FE5005D8F2E8E2D8D2C8C2BD20E8016D20180CE
:102FF50012D204800EC209800AE4F52AF5290528B3
:08300500022E310527022E08FE
:01300D0022A0
:1033B300C228C20CC208C207C205E4906837F0C233
:1033C3000F9066167405F0C22AE4F508FF7F40905B
:1033D30061B9E4F0A3DFFCE4FF7F20906617E4F01B
:1033E300A3DFFCE4FF74042FF582E43466F583E481
:1033F300F0740C2FF582E43466F583E4F00FBF0814
:10340300E4E4F50DF50EF512F511906302F0906307
:1034130001F0C203C20DC206C202C20AF50C9061DA
:1034230085F0F509F50BF55EC200C20B90683874A0
:10343300FFF0A374F4F0E4906403F0C20EC201C27F
:1034430004D209906EDDF0123876EF6003122E0578
:10345300E4F5137E617F87906186E0F513E513C37E
:1034630094014007E513D394084003E4F513E513EF
:1034730060220FEFAC0670010E14F5828C8374C4C6
:10348300F015130FEFAC0670010E14F5828C83E573
:1034930013F080DA906101E0F513E513C394014062
:1034A30007E513D394084003E4F513E51360220FF3
:1034B300EFAC0670010E14F5828C8374C8F01513FB
:1034C3000FEFAC0670010E14F5828C83E513F080C8
:1034D300DA906100E0F513E513C394014007E513A7
:1034E300D394084003E4F513E51360220FEFAC0611
:1034F30070010E14F5828C8374C2F015130FEFACB8
:103503000670010E14F5828C83E513F080DA0FEF59
:10351300AC0670010E14F5828C83E4F08F828E83E7
:10352300F0F513F59BC2ADF5C9D2CDD2CCC2C9C259
:10353300CAF5CDF5CC906838E0F5CBA3E0F5CA85A4
:10354300CBCD85CACCD29ED29CD2CAC2ACC298C2C1
:093553009975B81075B710D2ACDF
:01355C00224C
:1051F500E5106FFF90167093650FF510EF90157021
:0352050093F50F0F
:015208002283
:024371008F2D8E
:10437300E4FC752E61752F02F510F50FFDEDC39565
:104383002D5017052FE52FAE2E7002052E14F58242
:104393008E83E0FF1251F50D80E3052FE52FAE2E3E
:1043A3007002052E14F5828E83E510F0852F828529
:1043B3002E83E50FF0052D052D7E677F37752E6162
:1043C300752F028F828E837402F00FBF00010E0CD3
:1043D300E4FDEDC3952D5038852F82852E83E0F9BA
:1043E30064026008E964036003B9090D8F828E8358
:1043F3007409F00FBF00010E0C8F828E83E9F00F5A
:10440300BF00010E0C052FE52F7002052E0D80C293
:0F4413008F828E837403F00FBF00010E0CAF0475
:014422002277
:03527E00C2062243
:104ECD008F2C20033AAF2C124371906185EFF020A7
:104EDD001A127E147FA7123E4E7E617F02E4FBAD57
:104EED002C12429D300B057F011251B6E50960036E
:104EFD00F55B22E4F50CD203C2992099FDD29922DB
:022B64008F28B8
:102B6600E54724BE7003022DAD24FA7003022D271B
:102B760024046003022E04E54830E703022C2B30C0
:102B86001B077E147FB3123E4EE54A6068E549C3D3
:102B960094024003022E04E5497007E54A14F5291C
:102BA6008006E54A241FF529E52975F004A42403C7
:102BB600F582746335F0F5837D4C7F041232CAE5E5
:102BC6002975F004A42401F582746235F0F5837D3D
:102BD600507F041232CA74F92549F582E43461F54E
:102BE600837481F074B92529F582E43461F5837420
:102BF60001F0D20722301B077E147FBE123E4E74B0
:102C0600042549F582E43466F5837401F0E54975D7
:102C1600F004A42417F582746635F0F5837D4C7FA5
:102C2600041232CA22E54B64086003022E04E54909
:102C3600C394044003022E04301B077E147FC8127F
:102C46003E4E752801E54A5407FFE528A807088087
:102C560002C333D8FCF5287408250EF50EB50D060B
:102C66007408250DF50DE54A547FFFE549C4335434
:102C7600E02FFE7400250EF582E43460F583EEF055
:102C8600E54AC394805022EF131313541FFFE549FE
:102C960025E025E02F2417F582E43466F583E0FF6E
:102CA600E528F4FEEF5EF0802EE54A547FFF13130D
:102CB60013541FFFE54925E025E02F2417F582E48C
:102CC6003466F583E04528F07400250EF582E43479
:102CD60060F583E04480F07401250EF582E43460EB
:102CE600F5837D4C7F041232CAE551FEE550FF7C28
:102CF600007D0A1228E4EF7405250EF582E434609F
:102D0600F583EFF07406250EF582E43460F583E56D
:102D160052F07407250EF582E43460F583E553F02E
:102D260022301B077E147FCC123E4EE54A54E064E7
:102D3600407003022E04E549701DE54A1313543F03
:102D4600FF7401A807088002C333D8FC42119063C0
:102D560001E04511F08024E54964016003022E0478
:102D6600E54A1313543FFF7401A807088002C333D2
:102D7600D8FC4212906302E04512F0E54975F02056
:102D8600A4FFE54A547F7C002FFFEC35F0FEEF25CB
:102D9600E0FFEE33FE74042FF58274643EF5837D06
:102DA6004CAF4B1232CA22E54AB40113301B077EE0
:102DB600147FD1123E4EE54D04906FF6F0C228E521
:102DC6004AB40216240CF582E43466F583E54DF028
:102DD600301B077E147FD8123E4EE54AB4031F24EB
:102DE6000CF582E43466F583E54DF0301B077E145E
:0E2DF6007FE1123E4E302806906FDE7402F030
:012E040022AB
:10002600906403E070030208E630102F050A90661C
:1000360016E0600214F0906837E0600214F0C21017
:10004600302818906184E004F0E0D3940A400C3024
:100056001B077E147FE9123E4EC228E55BB4010EF3
:10006600E4F55BF50CD203C2992099FDD2993003D1
:100076000DE50AD394064009C203D20D8003E4F5C8
:100086000A300D0AC20D300B05E4FF1251B63003DB
:1000960003020542E55B6003020542200E062005C9
:1000A60003020542C205300F29C20FE4906102F037
:1000B600A37408F0906403E0906104F0906615E084
:1000C600906105F0A374FEF0A3748FF07F06124EC4
:1000D600CD22906FF6E0FF6025E4906102F0A374F4
:1000E60008F0906403E0906104F0A37483F0A3EF3A
:1000F600F0E4A3F0906FF6F07F06124ECD22E50EE7
:10010600650D7003020205906837E060030202DFA6
:10011600E50D2408F528E4906102F0A37408F09038
:100126006403E0906104F0A374F0F0A37406F0A3F6
:100136007491F074062528F582E43460F583E09026
:100146006108F074072528F582E43460F583E090B1
:100156006109F074012528F582E43460F583E090A6
:10016600610AF074022528F582E43460F583E09094
:10017600610BF074032528F582E43460F583E09082
:10018600610CF074042528F582E43460F583E09070
:10019600610DF074002528F582E43460F583E0FFF4
:1001A600547FFEC39440500BEFC454F00490610E8C
:1001B600F0801674002528F582E43460F583E0FFAC
:1001C600C454F0240590610EF074002528F582E4ED
:1001D6003460F583E0FFEEC4540F90610FF0EF54E6
:1001E60080FF74052528F582E43460F583E02F90BE
:1001F6006110F09068377414F07F0F124ECD2230E4
:10020600086AE4906102F0A37408F0906403E09039
:100216006104F0A37441F0A37420F0752A61752B74
:1002260007E4F52874172528F582E43466F583E09B
:10023600F529300906FF1251E18F29852B82852A7F
:1002460083E529F0F4FFE5822408F582E43583F599
:1002560083EFF0052BE52B7002052A0528E528C358
:10026600940840C07F15124ECDC20822300C6AE4B5
:10027600906102F0A37408F0906403E0906104F0CA
:10028600A37445F0A37420F0752A61752B077528B1
:100296000874172528F582E43466F583E0F52930DD
:1002A6000906FF1251E18F29852B82852A83E529CC
:1002B600F0F4FFE5822408F582E43583F583EFF058
:1002C600052BE52B7002052A0528E528C394104066
:1002D600C07F15124ECDC20C222007030203E29006
:1002E60061FAE0FF9061F9E04F5401D394005003A6
:1002F6000203E2E4F52874B92528F582E43461F5B1
:1003060083E070030203D474B92528F582E43461CE
:10031600F583E4F0906102F0A37408F0906403E0C2
:10032600906104F0A374F0F0A37403F0A37491F049
:10033600E528C4540F2408A3F0E528540FA3F0E5DC
:100346002825E025E0F5282401F582E43462F583CA
:10035600E090610AF074022528F582E43462F583A0
:10036600E090610BF074032528F582E43462F5838E
:10037600E090610CF074042528F582E43462F5837C
:10038600E090610DF0E4A3F074032528F582E434CF
:1003960063F583E090610FF074042528F582E43458
:1003A60063F583E0906110F074052528F582E43446
:1003B60063F583E0906111F074062528F582E43434
:1003C60063F583E0906112F07F11124ECD2205286D
:1003D600E528C3944050030202FCC207906616E06B
:1003E600704130043E7478F0E4906102F0A3740822
:1003F600F0906403E0906104F0A374F0F0E4A3F0DD
:10040600A37490F0A37408F0E4A3F0A3F0A3F0A300
:10041600F0A3F0A3F0A3F0A3F0A3F0A3F07F1112D2
:100426004ECD22E508C39404506FE50825E0FF741D
:1004360003A807088002C333D8FCF52855116528A0
:100446007053E528F45211E4906102F0A37408F0A9
:10045600906403E0906104F0A374F0F0A37402F0DA
:10046600A37491F0E5082420A3F0E5083333335450
:10047600F875F002A42404F582E5F03464F583638C
:10048600A20190610963A2017F101232DC7F17126C
:100496004ECD0508220508808AE508C394085076E3
:1004A600E50824FC25E0FF7403A807088002C3338F
:1004B600D8FCF528551265287058E528F45212E440
:1004C600906102F0A37408F0906403E0906104F078
:1004D600A374F0F0A37402F0A37491F0E50854033A
:1004E6002440A3F0E50833333354F875F002A4240E
:1004F60004F582E5F03464F58363A2019061096333
:10050600A2017F101232DC7F17124ECD0508530868
:10051600072205088083E4F508200E20E490610296
:10052600F0A37408F0906403E0906104F0A3749063
:10053600F0E4A3F0A3F07F06124ECD22906614E0FD
:10054600FF70030208E6F529E4F0201A1F7E147FE7
:10055600F7123E4EE52954802437F582E43466AF1F
:1005660082FEE529547FFDE4FB12429DE5297003D6
:100576000208E6E5295480FF2437F582E43466ADA7
:1005860082F52A8D2BE4F510F50F8F28E528C39503
:10059600295018052BE52BAE2A7002052A14F58280
:1005A6008E83E0FF1251F5052880E1E50F451060C6
:1005B6000E301A030208E67E157F00123E4E22E533
:1005C6002954802437F582E43466AF82F52A8F2BCE
:1005D6007402252BF52BE4352AF52A852B82F58323
:1005E600E0FF906403E0FEEF6E600E301A0302082F
:1005F600E67E157F0A123E4E22052BE52B7002057C
:100606002AF582852A83E0FFB43003D20522EF64FF
:100616000170030208E6EF64187037906605E0FF84
:10062600906604E04F600CD208201A077E157F1BE7
:10063600123E4E906607E0FF906606E04F7003029A
:1006460008E6D20C301A030208E67E157F24123E15
:100656004E22852B82852A83E0B41915201A077E3F
:10066600157F2D123E4E906301E0F511A3E0F512C1
:1006760022852B82852A83E0FF54F064F060030212
:10068600076E906615EFF0052BE52B7002052AF52F
:1006960082852A83E0FF64807033052BE52B700288
:1006A600052AF582852A83E0644060030208E6D2C3
:1006B6000F052BE52B7002052AF582852A83E06457
:1006C6000860030208E6D204906616F022EFB40131
:1006D60027052BE52B7002052AF582852A83E0641F
:1006E6004F60030208E6906837E070030208E6747C
:1006F60008250DF50DE4F022852B82852A83E0601E
:10070600030208E6052BE52B7002052AF582852AE9
:1007160083E0644260030208E6052BE52B700205C0
:100726002AF582852A83E0906FE0F0052BE52B7091
:1007360002052AF582852A83E0906FE1F0052BE514
:100746002B7002052AF582852A83E0906FE2F00578
:100756002BE52B7002052AF582852A83E0906FE34C
:10076600F0D22AC204D20F22852B82852A83E0FF8B
:1007760064116008EF641260030208C4E529547F1F
:10078600640E60030208C4201A077E157F36123EE7
:100796004E30280E301A030208E67E157F4B123EB5
:1007A6004E22852B82852A83E0540314F529052BD6
:1007B600E52B7002052AF582852A83E0F52830E7C5
:1007C60009E4906FDFF0906FE4F0E52830E60BE483
:1007D600906FDFF0906FE47410F0E52830E50B9031
:1007E6006FDF7401F0E4906FE4F0E52830E40C90DC
:1007F6006FDF7401F0906FE47410F0E52830E30BBE
:10080600906FDF7402F0E4906FE4F0E52830E20CBC
:10081600906FDF7402F0906FE47410F0E52830E119
:100826000B906FDF7403F0E4906FE4F0E52830E09E
:100836000C906FDF7403F0906FE47410F07402256F
:100846002BF52BE4352AF52A852B82F583E0F5284E
:1008560030E700E52830E607906FE4E02402F0E593
:100866002830E507906FE4E02404F0E52830E4073B
:10087600906FE4E02406F0E52830E307906FE4E0AB
:100886002408F0E52830E207906FE4E0240AF0E55A
:100896002830E107906FE4E0240CF0E52830E0070B
:1008A600906FE4E0240EF0906FE4E02529F0D22862
:1008B600E4906184F0906FDEF0906FF6F022201ADB
:1008C6001F7E157F59123E4EE52954802437F58246
:1008D600E43466AF82FEE529547FFDE4FB12429DB7
:0108E60022EF
:1047C7000217B0E493A3F8E493A34003F68001F241
:1047D70008DFF48029E493A3F85407240CC8C333F3
:1047E700C4540F4420C8834004F456800146F6DFC2
:1047F700E4800B0102040810204080905263E47E9D
:10480700019360BCA3FF543F30E509541FFEE493B6
:10481700A360010ECF54C025E060A840B8E493A37D
:10482700FAE493A3F8E493A3C8C582C8CAC583CAA8
:10483700F0A3C8C582C8CAC583CADFE9DEE780BE60
:015269000044
:10289E00BB010689828A83E0225002E722BBFE0238
:0928AE00E32289828A83E493226B
:1028B700BB010CE58229F582E5833AF583E02250D6
:1028C70006E92582F8E622BBFE06E92582F8E22220
:0D28D700E58229F582E5833AF583E493223A
:1028E400BC000BBE0029EF8DF084FFADF022E4CCD8
:1028F400F875F008EF2FFFEE33FEEC33FCEE9DECA1
:10290400984005FCEE9DFE0FD5F0E9E4CEFD22EDE6
:10291400F8F5F0EE8420D21CFEADF075F008EF2F30
:10292400FFED33FD4007985006D5F0F222C398FD21
:052934000FD5F0EA22BE
:1029390075F008758200EF2FFFEE33FECD33CDCC55
:1029490033CCC58233C5829BED9AEC99E5829840D8
:102959000CF582EE9BFEED9AFDEC99FC0FD5F0D6B5
:10296900E4CEFBE4CDFAE4CCF9A88222B800C1B9DF
:102979000059BA002DEC8BF084CFCECDFCE5F0CB1D
:10298900F97818EF2FFFEE33FEED33FDEC33FCEB56
:1029990033FB10D703994004EB99FB0FD8E5E4F911
:1029A900FA227818EF2FFFEE33FEED33FDEC33FCFE
:1029B900C933C910D7059BE99A4007EC9BFCE99AF2
:1029C900F90FD8E0E4C9FAE4CCFB2275F010EF2F37
:1029D900FFEE33FEED33FDCC33CCC833C810D70737
:1029E9009BEC9AE899400AED9BFDEC9AFCE899F872
:0E29F9000FD5F0DAE4CDFBE4CCFAE4C8F92205
:0E2A0700C3E49FFFE49EFEE49DFDE49CFC22E0
:102A1500EB9FF5F0EA9E42F0E99D42F0E89C45F017
:012A2500228E
:0C2A2600ECF0A3EDF0A3EEF0A3EFF02223
:102A3200A8828583F0D083D082122A49122A4912B1
:102A42002A49122A49E473E493A3C583C5F0C583D6
:102A5200C8C582C8F0A3C583C5F0C583C8C582C8EE
:012A62002251
:10227300E53B242FF8E6053B22782C302602782F05
:10228300E475F001122AC402289E201FEB7F2ED290
:102293001F8018EF540F2490D43440D4FF30230B05
:1022A300EF24BFB41A0050032461FFE53C6002151C
:1022B3003C053FE53F7002053E30260D782CE47562
:1022C300F001122AC4EF022A63024DB87403D22626
:1022D3008003E4C226F53B8B2C8A2D892EE4F53C42
:1022E300F53EF53FE53C60077F201222AE80F57591
:1022F3003DFFC220C21FC221C222C224C225C2275F
:1023030012227CFF700D3026057F001222BFAF3FE3
:10231300AE3E22B4255FC2D5C22312227CFF24D055
:10232300B40A00501A75F00A783C30D50508B6FF98
:102333000106C6A426F620D5047002D22280D92431
:10234300CFB41A00EF5004C2E5D2230224BFD22037
:1023530080C6D21F80C0D22180BCD2D580BAD224FD
:1023630080B47F201222AE2021077401B53C0040C7
:10237300F1122273FF1222AE0222E7D227D2258066
:1023830095122273FB122273FA122273F94A4B70CD
:102393000679907A257BFF20212EE53C602A7E007A
:1023A3008E827583001228B760060EEE653D70F0CD
:1023B300C2D5EBC0E0EAC0E0E9C0E0EE122506D0EA
:1023C300E0F9D0E0FAD0E0FB12289EFF60AAEBC050
:1023D300E0EAC0E0E9C0E01222AED0E02401F9D087
:1023E300E03400FAD0E0FBE53D0460DCD53DD98064
:1023F300877BFF7A257902D221809C79108002792C
:1024030008C225C2278008D2D5790A8004790AC276
:10241300D5E53D047002F53DE4FAFDFEFF1222739B
:10242300FC7B08202013122273FD7B10301F0A123D
:102433002273FE122273FF7B20EC3382D592D55098
:1024430013C3E4301F069FFFE49EFEE42020039D98
:10245300FDE49CFCE4CBF8C220EC700CCFCECDCCD9
:10246300E824F8F870F38017C3EF33FFEE33FEED83
:1024730033FDEC33FCEB33FB994002FB0FD8E9EB64
:10248300302005F8D0E0C448B220C0E00AEC4D4E3D
:102493004F78207B0070C2EAB53D0040BCC0E0121B
:1024A3002508D0F0D0E0202004C4C0E0C4B220C08E
:1024B300F0122297D0F0D5F0EB0222E7122B232360
:1024C300845323FE5823554C23514224024F240A9C
:0F24D30044240A49236A4324105523F44623F472
:1024E2004523F44725B05023592D235D2E23802BFD
:1024F200236123237E2025992A231948000023786B
:102502003F3F3F00790AA2D5202214302409B91096
:10251200020404B9080104A2D520250250010420B6
:1025220021689221B53C005034C0E07F203022194E
:102532007F30A22172257224500F12255FC221C260
:1025420025C224C2277F30800F302403E9C0E01265
:1025520022AE302403D0E0F9D0E0B53CCC302417D1
:102562007F30B9100C1222AE7F583023077F78805B
:1025720003B908031222AE3021057F2D0222AE7F5D
:10258200202027F87F2B2025F322922180CF286E4E
:10259200756C6C2900D2201222733020F8C2207888
:1025A2003C30D50108F60223192D50434958122216
:1025B200732403B405004001E49025AB9312229FDB
:0D25C200743A12229FD222753C040223FEBF
:10355D008B2F8A308931E4F53BF53AF539F538F59D
:10356D0036F537E533453445326012EBC0E0EAC03D
:10357D00E0E9C0E0AB32AA33A934122AD4AB2F054F
:10358D0031E531AA307002053014F912289EF53C50
:10359D00C394094007E53CD3940D40E1E53C64201C
:1035AD0060DBE53CB42D054337038016E53CB42BB9
:1035BD0005433701800C74FF2531F53174FF35302B
:1035CD00F530E53560046410703FAB2FAA30A9319A
:1035DD0012289E64306009E535702E75350A8029F4
:1035ED009000011228B7FF64786004EFB4581343BC
:1035FD00370175351074022531F531E43530F5306C
:10360D008007E5357003753508AB2F0531E531AA17
:10361D00307002053014F912289EF53CC3946140B8
:10362D000AE53CD3947A5003533CDF74D0253CF526
:10363D003CC3940A400CE53C9411406D74F9253C53
:10364D00F53CE53CD395355060433701853B4085CE
:10365D003A3F85393E85383DAF357E00E4FCFDAB04
:10366D003BAA3AA939A838122A75C8ECC8C9EDC9C0
:10367D00CAEECACBEFCBE4FCFDFEEB253CF53BEEF1
:10368D003AF53AED39F539EC38F538AF3BAE3AADA0
:10369D0039FCAB40AA3FA93EA83DD3122A155003D1
:1036AD00023616433704023616E53720E003E48070
:1036BD002DE53345344532601EAB2FE53124FFF93E
:1036CD00E53034FFFAEBC0E0EAC0E0E9C0E0AB3230
:1036DD00AA33A934122AD4E53730E20774FFFFFE6E
:1036ED00FDFC22E537AF3BAE3AAD39AC3830E103E6
:0436FD00022A072274
:102A6300BB010689828A83F0225002F722BBFE0152
:022A7300F3224C
:102A7500E88FF0A4CC8BF0A42CFCE98EF0A42CFC00
:102A85008AF0EDA42CFCEA8EF0A4CDA8F08BF0A47E
:102A95002DCC3825F0FDE98FF0A42CCD35F0FCEBDD
:102AA5008EF0A4FEA9F0EB8FF0A4CFC5F02ECD39A2
:0F2AB500FEE43CFCEAA42DCE35F0FDE43CFC220F
:102AC400FAE6FB0808E6F925F0F618E6CA3AF62213
:102AD400BB011A89828A83D0F0D0E0F8D0E0F9D023
:102AE400E0FAD0E0FBE8C0E0C0F0022B525016E957
:102AF400F8D083D082D0E0F9D0E0FAD0E0FBC082F5
:102B0400C083022B49BBFE16E9F8D083D082D0E003
:0F2B1400F9D0E0FAD0E0FBC082C083022B5B2235
:102B2300D083D082F8E4937012740193700DA3A341
:102B330093F8740193F5828883E473740293686055
:062B4300EFA3A3A380DF55
:092B4900EBF608EAF608E9F622B1
:092B5200EBF0A3EAF0A3E9F02284
:092B5B00EBF208EAF208E9F222AB
:00000001FF
